:020000040000fa
:08000000101b040000000000c9
:020000040000fa
:10000800041a0000081a00000c1a0000101a000058
:10001800141a00000c1b00000c1b00000c1b000035
:10002800181a00001c1a0000201a0000241a0000e8
:100038000c1b0000281a00002c1a0000301a0000bf
:10004800341a0000381a00003c1a0000401a000058
:10005800441a0000481a00000c1b00000c1b00008a
:100068004c1a0000501a0000541a0000581a0000d8
:100078005c1a00000c1b0000601a0000641a0000e3
:100088000c1b0000681a00006c1a0000701a0000af
:10009800741a0000781a00007c1a0000801a000008
:1000a800841a0000881a00000c1b00000c1b0000ba
:1000b8000c1b00008c1a0000901a0000941a000013
:1000c800981a00009c1a0000a01a0000a41a000048
:1000d800a81a0000ac1a00000c1b00000c1b000042
:1000e8000c1b0000b01a0000b41a00000c1b000022
:1000f8000c1b0000b81a0000bc1a00000c1b000002
:100108000c1b00000c1b00000c1b00000c1b00004b
:100118000c1b00000c1b0000c01a00000c1b000088
:100128000c1b0000c41a0000c81a0000cc1a0000fa
:100138000c1b00000c1b00000c1b00000c1b00001b
:10014800d01a00000c1b00000c1b00000c1b000048
:100158000c1b0000d41a00000c1b00000c1b000034
:100168000c1b0000d81a0000dc1a0000e01a00007e
:10017800e41a0000e81a0000ec1a0000f01a000067
:10018800f41a0000f81a0000fc1a0000001b000016
:10019800041b0000081b00000c1b00000c1b0000c7
:1001a8000c1b00000c1b00000c1b00000c1b0000ab
:1001b8000c1b00000c1b00000c1b00000c1b00009b
:1001c8000c1b00000c1b00000c1b00000c1b00008b
:1001d8000c1b00000c1b00000c1b00000c1b00007b
:1001e8000c1b00000c1b00000c1b00000c1b00006b
:0801f8000c1b00000c1b0000b1
:020000040000fa
:04020800ec1b0000eb
:020000040000fa
:04020c00ec1b0000e7
:020000040000fa
:04021000ec1b0000e3
:020000040000fa
:04021400ec1b0000df
:020000040000fa
:04021800ec1b0000db
:020000040000fa
:04021c00ec1b0000d7
:020000040000fa
:04022000ec1b0000d3
:020000040000fa
:04022400ec1b0000cf
:020000040000fa
:04022800ec1b0000cb
:020000040000fa
:04022c00ec1b0000c7
:020000040000fa
:04023000ec1b0000c3
:020000040000fa
:04023400ec1b0000bf
:020000040000fa
:04023800ec1b0000bb
:020000040000fa
:04023c00ec1b0000b7
:020000040000fa
:04024000ec1b0000b3
:020000040000fa
:04024400ec1b0000af
:020000040000fa
:04024800ec1b0000ab
:020000040000fa
:04024c00ec1b0000a7
:020000040000fa
:04025000ec1b0000a3
:020000040000fa
:04025400ec1b00009f
:020000040000fa
:04025800ec1b00009b
:020000040000fa
:04025c00ec1b000097
:020000040000fa
:04026000ec1b000093
:020000040000fa
:04026400ec1b00008f
:020000040000fa
:04026800ec1b00008b
:020000040000fa
:04026c00ec1b000087
:020000040000fa
:04027000ec1b000083
:020000040000fa
:04027400ec1b00007f
:020000040000fa
:04027800ec1b00007b
:020000040000fa
:04027c00ec1b000077
:020000040000fa
:04028000ec1b000073
:020000040000fa
:04028400ec1b00006f
:020000040000fa
:04028800ec1b00006b
:020000040000fa
:04028c00ec1b000067
:020000040000fa
:04029000ec1b000063
:020000040000fa
:04029400ec1b00005f
:020000040000fa
:04029800ec1b00005b
:020000040000fa
:04029c00ec1b000057
:020000040000fa
:0402a000ec1b000053
:020000040000fa
:0402a400ec1b00004f
:020000040000fa
:0402a800ec1b00004b
:020000040000fa
:0402ac00ec1b000047
:020000040000fa
:0402b000ec1b000043
:020000040000fa
:0402b400ec1b00003f
:020000040000fa
:0402b800ec1b00003b
:020000040000fa
:0402bc00ec1b000037
:020000040000fa
:0402c000ec1b000033
:020000040000fa
:0402c400ec1b00002f
:020000040000fa
:0402c800ec1b00002b
:020000040000fa
:0402cc00ec1b000027
:020000040000fa
:0402d000ec1b000023
:020000040000fa
:0402d400ec1b00001f
:020000040000fa
:0402d800ec1b00001b
:020000040000fa
:0402dc00ec1b000017
:020000040000fa
:0402e000ec1b000013
:020000040000fa
:0402e400ec1b00000f
:020000040000fa
:0402e800ec1b00000b
:020000040000fa
:0402ec00ec1b000007
:020000040000fa
:0402f000ec1b000003
:020000040000fa
:0402f400ec1b0000ff
:020000040000fa
:0402f800ec1b0000fb
:020000040000fa
:0402fc00ec1b0000f7
:020000040000fa
:04030000ec1b0000f2
:020000040000fa
:04030400ec1b0000ee
:020000040000fa
:04030800ec1b0000ea
:020000040000fa
:04030c00ec1b0000e6
:020000040000fa
:04031000ec1b0000e2
:020000040000fa
:04031400ec1b0000de
:020000040000fa
:04031800ec1b0000da
:020000040000fa
:04031c00ec1b0000d6
:020000040000fa
:04032000ec1b0000d2
:020000040000fa
:04032400ec1b0000ce
:020000040000fa
:04032800ec1b0000ca
:020000040000fa
:04032c00ec1b0000c6
:020000040000fa
:04033000ec1b0000c2
:020000040000fa
:04033400ec1b0000be
:020000040000fa
:04033800ec1b0000ba
:020000040000fa
:04033c00ec1b0000b6
:020000040000fa
:04034000ec1b0000b2
:020000040000fa
:04034400ec1b0000ae
:020000040000fa
:04034800ec1b0000aa
:020000040000fa
:04034c00ec1b0000a6
:020000040000fa
:04035000ec1b0000a2
:020000040000fa
:04035400ec1b00009e
:020000040000fa
:04035800ec1b00009a
:020000040000fa
:04035c00ec1b000096
:020000040000fa
:04036000ec1b000092
:020000040000fa
:04036400ec1b00008e
:020000040000fa
:04036800ec1b00008a
:020000040000fa
:04036c00ec1b000086
:020000040000fa
:04037000ec1b000082
:020000040000fa
:04037400ec1b00007e
:020000040000fa
:04037800ec1b00007a
:020000040000fa
:04037c00ec1b000076
:020000040000fa
:04038000ec1b000072
:020000040000fa
:04038400ec1b00006e
:020000040000fa
:04038800ec1b00006a
:020000040000fa
:04038c00ec1b000066
:020000040000fa
:04039000ec1b000062
:020000040000fa
:04039400ec1b00005e
:020000040000fa
:04039800ec1b00005a
:020000040000fa
:04039c00ec1b000056
:020000040000fa
:10340000101b040000000000ec1b04000000000082
:10341000ec1b040000000000ec1b04000000000096
:10342000ec1b040000000000ec1b04000000000086
:10343000ec1b040000000000ec1b04000000000076
:10344000ec1b040000000000d81b0400000000007a
:10345000ec1b040000000000ec1b04000000000056
:10346000ec1b040000000000ec1b04000000000046
:10347000ec1b040000000000ec1b04000000000036
:10348000ec1b040000000000ec1b04000000000026
:10349000ec1b040000000000ec1b04000000000016
:1034a000ec1b040000000000ec1b04000000000006
:1034b000ec1b040000000000ec1b040000000000f6
:1034c000ec1b040000000000ec1b040000000000e6
:1034d000ec1b040000000000ec1b040000000000d6
:1034e000ec1b040000000000ec1b040000000000c6
:1034f000ec1b040000000000ec1b040000000000b6
:10350000ec1b040000000000ec1b040000000000a5
:10351000ec1b040000000000ec1b04000000000095
:10352000ec1b040000000000ec1b04000000000085
:10353000ec1b040000000000ec1b04000000000075
:10354000ec1b040000000000ec1b04000000000065
:10355000ec1b040000000000ec1b04000000000055
:10356000ec1b040000000000ec1b04000000000045
:10357000ec1b040000000000ec1b04000000000035
:10358000ec1b040000000000ec1b04000000000025
:10359000ec1b040000000000ec1b04000000000015
:1035a000ec1b040000000000ec1b04000000000005
:1035b000ec1b040000000000ec1b040000000000f5
:1035c000ec1b040000000000ec1b040000000000e5
:1035d000ec1b040000000000ec1b040000000000d5
:1035e000ec1b040000000000ec1b040000000000c5
:1035f000ec1b040000000000ec1b040000000000b5
:10360000ec1b040000000000ec1b040000000000a4
:10361000ec1b040000000000ec1b04000000000094
:020000040000fa
:103620004f8d20000e7f24000e0188000000000056
:10363000000020000000e000020032000001200035
:103640002002880014000700650007000000e00069
:1036500003003a0060ca2200010020000200370087
:103660000000200001002000810f700001003200e6
:1036700014000700000020000000e00002003200fb
:1036800000000200000000004c2a020000000000c0
:103690000040da000000fe004440a9008005200040
:1036a0000000e0000300320000002000a0018800bc
:1036b0004440a800000006008a1f78008b1f780095
:1036c0000000060091018800800478000000eb00f3
:1036d0001a003700e284440032a0b4009905ba0011
:1036e000e284440032a0b4009906ba00e2844400a7
:1036f00032a0b4000006eb00476fde00fd07b20009
:10370000636ce10003003a00ebff07000000eb00f0
:103710000a003700606ce10004003a00005deb0035
:103720008b05e900fdff3e00040037006168e10001
:10373000010032000086eb000b00070019c7ba0039
:103740001905ba000e04e00003003a000a00e00088
:10375000e0ff3a0000000600fe07b2009e0188006c
:103760008a047800f5ff3700395dba008b05e9005f
:103770000c003200295dba008b05e9000800320018
:103780000c00e00003003a00e284440032a0b400e0
:10379000f5ff370019ddba008b05e900faff3a00a2
:1037a0008904e800e184440032a0b400000006006f
:1037b0003400f800881f780008002000a801880065
:1037c0004f0478000000fa008460a9000080fa002d
:1037d0003400f900004006000040da000000fe005e
:1037e000000005000000fa0068815700cfb897007c
:1037f000460207000080fa00000006006a00070089
:10380000c2000700730107009b010700f4000700d6
:103810009602070041023700889fbe008a9fbe00c3
:10382000800478000200e0005b0032000140780074
:10383000814c780082814400f1f99f00e20f510031
:103840005500360091449800a1449800e1f99f008a
:10385000d1f99f00e60f51004f003600b1449800a7
:10386000c1f99f00e80f51004b0036000905ea003e
:10387000630565000a8444000a055100c1ff2f005a
:10388000010565000080fb008000eb0012102000a5
:103890001310200082050700008cbe000a014400be
:1038a00060b99f0071b99f00e80f55003a003600db
:1038b00020049800310498004004980051049800b6
:1038c00020b99f0031b99f0040b99f0051b99f00b6
:1038d000f80f55003000360060049800710498001d
:1038e000000c9800110c9800200c9800310c9800e6
:1038f000400c9800510c980020b19f0031b19f00fe
:1039000040b19f0051b19f0060b19f0071b19f0015
:1039100000b99f0011b99f00640164007801410063
:1039200002044400020555006011b8000203be0005
:103930000002be000403be006022b8000000720056
:1039400081807200020173008381730010003700d0
:10395000009cbe000294be004004980051049800f0
:103960006204980073049800000c9800110c9800f1
:10397000220c9800330c9800400c9800510c9800d1
:10398000620c9800730c98000a02b1000802b000a3
:10399000ff0f5500eeff3e00090078004f05be0006
:1039a0004f04be0000000600ec874700889fbe0061
:1039b0008a9fbe008c9fbe008e1f78000006780094
:1039c00001047800180790002805900098067800f8
:1039d000cdb79f00b80590003202be002203be00a2
:1039e0000400be000601be004f18de006011b800e2
:1039f0008000eb00d0b79f00e1b79f00f2b79f00b7
:103a000083bf9f00800478000900e00006003200b8
:103a10006000b8006011b8000402500085825800b0
:103a200006035900878359000e00e00002003500ac
:103a30000d10a100cdb79f000900e00005003a007d
:103a40004fb097000028a30002003a000038a300fe
:103a5000020032008a00e900010037008a00780085
:103a6000f8815700a20020000800780086000700b7
:103a70000900e00003003a00cfb097000128a3003e
:103a8000080032000000e90000814500b1c2b30027
:103a90000900e00001003200d1c2b3000149780002
:103aa000050037000138a300030032000000e900e0
:103ab00001c2b30081757800480190000201e9005d
:103ac00000015100808045004fb297008a017800c4
:103ad0000c007800300207009c0090000188a300d1
:103ae0000400320098009000810f500001003d005a
:103af000010078004f0778004f06be004f05be005a
:103b00004f04be00cf00b100000006000200fa0022
:103b1000889fbe008a9fbe0080057800010478005f
:103b200002007800180190002805900098007800a5
:103b3000b1bf9f00b80490000200e0000200350011
:103b40000110a100b1bf9f00ea8157008200200050
:103b50008a0078003002be002003be000800780012
:103b6000490007003fb99700f000610003003200f0
:103b70000000e90001c3b300817478003fb99700e9
:103b8000e8006100030032000000e90001c2b30058
:103b900081747800480190000201e90000015100a1
:103ba000808044003fba97008a0178000b007800bb
:103bb000f90107009b0090000188a3000400320077
:103bc00098009000810f500001003d000100780036
:103bd0004f05be004f04be000080fa000000060042
:103be000ea874700889fbe008a9fbe008e1f78002c
:103bf00000047800030078007287570084e22600f2
:103c000055c72600049fbe00c3962200030f78000c
:103c10006c875700004feb0011059000a104900045
:103c2000910578000200e0000200320002077800ef
:103c300001003700728757000000e00002003a00e0
:103c40000e007800ea0307000a00e00003003500d8
:103c50008a0f5000010036000a0078000b0278003d
:103c600089017800000178008e0078000800780053
:103c7000c90107004f0778004f05be004f04be0082
:103c8000af00b10000000600f4874700889fbe0027
:103c90008a9fbe008c9fbe008e1f78000605be0066
:103ca0000404be0081bf9f0082b79f00f3b79f004e
:103cb000b0009000e1b79f001301780092b79f0019
:103cc00090069000400090000000e9000006780097
:103cd0000d00e00001003d001d0020008040eb00d1
:103ce000efb19700817178001e0020001f0037009f
:103cf0000c06e9000fb09700cf80de006109b90023
:103d0000a0b79f00b1b79f00c2b79f00d3b79f0075
:103d10000203be000002be000800be000a01be0091
:103d200005050700000778000e4078000043b0004a
:103d3000efb0970080707e008d06e9000fb9970004
:103d40000201e90082bf9f002fb29700bfb2970027
:103d50004fb39700dfb397000800be000a01be0012
:103d6000ee0407000205be000004be000c00e000e7
:103d70000d003400e00f5400e08f5c00e00f5d00a8
:103d8000e08f5d00daff3a000d00e000d8ff3c0054
:103d90008fb997000300e000030034001fb09700c4
:103da0000018a300d2ff3a000e00e00002003a0023
:103db000ffb097001140a1000c0078004f07780079
:103dc0004f06be004f05be004f04be004f01b100bc
:103dd000000006000200fa00889fbe008a9fbe0015
:103de00000057800010478000200780018019000b6
:103df000a804900098007800b1bf9f00b80590001b
:103e00000200e000020035000110a100b1bf9f00d8
:103e1000ea815700a2002000890078003002be002d
:103e20002003be000800780097ff070048019000bb
:103e30000201e90000015100808045003fba97006f
:103e4000890178000a007800530107009a00900069
:103e50000188a3000400320098009000810f5000f8
:103e600001003d00010078004f05be004f04be0078
:103e70000080fa0000000600fa874700889fbe0015
:103e80008a9fbe008c9fbe008e1f78008004780041
:103e90000104780082057800180190002805900040
:103ea00018077800b80090000200e000020035001a
:103eb0000e10a10001003700120020007000670002
:103ec000e0b79f00090032003b02be002b03be009a
:103ed000e00f5200e08f5a00e00f5b00e08f5b00c4
:103ee000020032008a86e900010037008a06780065
:103ef000e8026700f5b79f00010032008d06e90077
:103f00003b02be002b03be00e4af9f00f5af9f0055
:103f100086b79f0097b79f00480690000c06e900ff
:103f20000040eb0080707e00efb297007fb29700f8
:103f30008903780081047800d8af9f0002047800dc
:103f40008bbf9f008a057800034578002a00370060
:103f50000c06e9006fab97006f006300e90f50009b
:103f600002003c000003b000010037007005b00003
:103f70000a03fb001604b100f90f53000c003e00c9
:103f8000000378000650a0001606b100f90f530098
:103f900007003e00b4b79f00a5b79f00c7b79f00ba
:103fa00032030700cfb39700afb297003fb297003c
:103fb00080747e000804e9008d06e9006fa8970070
:103fc000ffa897000fb197009fb19700460020000f
:103fd0008301d1000281d3008180d3000080d3000f
:103fe0000603e900faff3a00e0af9f00f1af9f003f
:103ff00082b79f0093b79f00e10f56000f00340077
:104000006fa89700ffa897000fb197009fb1970086
:10401000e00f5000e08f5800e00f5900e08f59008a
:10402000cbff3a000800e000c9ff3c000d00e000b3
:10403000020034000e18a300c5ff3a008900780082
:10404000f4b79f00870478005fac97008a4178003e
:104050000b0578008fbd97000500e00010003200ce
:104060003b02be002b03be00e4af9f00f5af9f00f4
:1040700086b79f0097b79f00e00f5200e08f5a006d
:10408000e00f5b00e08f5b00050032000c06e900ea
:1040900083707e000c06e90000c3b30080707e00d0
:1040a000ffb297000500e000030032000c06e900b3
:1040b00000c2b30080707e00480190000201e90058
:1040c0000c0151008c8040000e0278008a017800bb
:1040d00009007800b0000700990090000188a30053
:1040e0000400320098009000810f500001003d0054
:1040f000010078004f0778004f06be004f05be0054
:104100004f04be00af01b10000000600820178003c
:1041100001017800f1ff2700db023700840820004e
:10412000848f50001d0032000d003c001408200058
:10413000848f50002700320002003c000408200059
:104140000400370024082000848f5000340032001f
:1041500044082000848f500043003a0036003700a6
:10416000040a2000848f50002700320004003c0025
:1041700004092000848f50003b003a0028003700db
:10418000020c2000828f50002f003200020f20000e
:10419000828f500034003a002b0037009380e900f2
:1041a0000200e00005003200810978001102fb00e6
:1041b000cfa2de00612bb90028003700810978000a
:1041c000114278000482fb008002eb006033b800eb
:1041d0002200370013027800e40052000200e000e1
:1041e00005003200810978001102be004fabde00ed
:1041f0008603780019003700810978001102be009b
:104200006033b800150037009380e9008109780019
:1042100011027800cfa2de00612bb9000f00370039
:1042200093027800e8805200810978003102be00d4
:104230002103be00090037009380e9000200e0007e
:1042400002003200f1ff37009380e9008109780015
:10425000110278008002eb006033b8000498be00c1
:104260000690be0010000500000005004408200074
:10427000848f50002500320008003c001408200004
:10428000848f50001400320024082000848f5000d6
:1042900024003200040820000c003700040920002c
:1042a000848f50001f00320004003c00840820006e
:1042b000848f500024003a000e003700040a2000ca
:1042c000848f500011003200040c2000848f5000b5
:1042d0001d003a000d0037009380e9008109780045
:1042e0009100780001087800cf91de008288be003e
:1042f000140037009380e90081097800910078006c
:1043000001087800824878000e0037009380e900a9
:10431000810978009100780001087800820878000f
:10432000080037009380e900810978009100780047
:10433000010878006112b900612bb9008498be00b1
:104340008690be001000050000000500889fbe009a
:10435000000478004800900082047800808f5400a8
:1043600001003600800478000901780058009000b0
:1043700018020700580090000900400050049800ff
:10438000c800900089845000490498000048eb0060
:104390004f04be0000000600f2874700889fbe0061
:1043a0008a9fbe008c9fbe008e1f7800800478001c
:1043b0000105780002047800830578006107620037
:1043c00002003a008b0f5400080039000801780001
:1043d0008a00780009007800dcff07008b0f54008a
:1043e00002003900880578001e0037000886550055
:1043f0000c017800f00f5600010036000201200089
:10440000010220007e80570003fd07008c06780023
:104410000500370002012000fe80570009007800e7
:10442000caff0700f0865600ef8f5600f9ff3e00e6
:104430004461de0000ff2f000091b9000201460038
:10444000fe80570009007800c0ff07000e00e00062
:1044500004003a00080178008a007800090078001a
:10446000baff07000b0078004f0778004f06be0028
:104470004f05be004f04be002f01b1000000060032
:1044800000000500000005000000050000017800a4
:104490000040eb008080fb0081804000838520008d
:1044a00063c278000404e00003003a009085200015
:1044b00060c078000000060092017800934f52001f
:1044c00004003a009085200060c078000309e800ed
:1044d000010037000040e800ea4f5000edff3600d1
:1044e00000000600f6874700889fbe008a9fbe0036
:1044f0008c9fbe008e1f78000005780001047800b4
:1045000083057800040678000000eb00c0b79f0028
:104510008080eb00d1b79f00e0b79f00f2b79f000b
:104520000008200080bf9f009800780001007800fc
:104530008004eb00010037008904e8003041780076
:104540000204e0000300320053c2b300834f510065
:10455000f9ff3a000900e000040032000901780088
:104560000a00780079ff0700188c440018077800cb
:1045700050c2b3009e4f10003f013a000e07e80002
:104580000e0c780010003700cfb097000100a0009b
:104590000b003700cfb097000110a00008003700d3
:1045a000cfb097000120a00005003700cfb09700e2
:1045b0000130a00002003700cfb097000140a000fa
:1045c000c1b79f00000ce800180078009040780008
:1045d000b2c2b30082cf5000f1ff320007003c00ae
:1045e00002c2b30082cf5000f0ff320032c2b300eb
:1045f00082cf500007003a00efff3700d2c2b3006d
:1046000082cf5000e0ff320002c3b30082cf5000df
:10461000e0ff3200a2c2b30082cf50000d003a008a
:10462000000ce8001c80e900000e78001000780003
:10463000e0b79f000000e0000f003d00cfb0970002
:104640000100a200c1b79f000000ea00e0b79f0090
:104650000900370039010700e0b79f00010037006b
:10466000000ce800180078009000fb000103b10086
:10467000e98f5000faff36004fb097000008a30002
:10468000020032000010a100c0b79f00180078009f
:10469000e1c2b30090cf100016003a008000eb009a
:1046a000d1b79f000000e800000c7800a1c2b30061
:1046b00090cf100006003a00000ce8001c80e900d2
:1046c000000e780010007800d0b79f000900370076
:1046d0001a010700d0b79f0001003700000ce80066
:1046e000180078009000fb000103b100e98f500032
:1046f000faff36000800780064ff07008046780063
:10470000180078001000fb005101070091062000fe
:10471000810f50003800320012003c00410620009a
:10472000810f5000340032000a003c0011062000c6
:10473000810f50002000320031062000810f500010
:10474000a000320051022000810f5000bc003a004e
:10475000b400370071062000810f5000b8003c0003
:104760008800370001072000810f50005c003200f4
:1047700007003c00e1062000810f50007a00320063
:10478000f1062000810f5000ad003a0039003700db
:1047900051072000810f50002700320081072000c0
:1047a000810f50004200320031072000810f50007d
:1047b000a3003a008f0037008d80fb000c017800c9
:1047c00000fe2f000f004000540107000000e00031
:1047d000a800320018007800000ce8009041780032
:1047e00002fe2f000f014100f88057000a007800f8
:1047f00024ff07000e0037008d80fb008c0178003d
:104800001200200000fe2f000f00400043fe0700b2
:104810000000e00097003200180ce80002fe2f00b4
:104820000f014100f88057000a0078005efc070085
:1048300080844400900037008d80fb008c0178005c
:104840000001eb0000fe2f000f00400033fe0700c8
:104850000000e00087003200180ce80002fe2f0084
:104860000f014100f88057000a00780059fd070049
:10487000efff37008d80fb008c0178000001eb001a
:1048800000fe2f000f00400024fe07000000e000a3
:1048900078003200180ce80002fe2f000f014100e2
:1048a000f88057000a00780098fc0700e0ff370006
:1048b0008d80fb008c0178000001eb0000fe2f00d2
:1048c0000f00400015fe07000000e0006900320004
:1048d00018007800000ce800904178001c003700b8
:1048e0008c0178000001eb00010f200000fe2f007a
:1048f0000f00400009fe07000000e0005d003200ec
:10490000180ce8000fb097009fb097002fb19700e8
:10491000bfb19700e00f5000e08f5800e00f590042
:10492000e08f590009003a00cfb597006fb49700a7
:1049300000852000ae0007000b0278008801780097
:1049400000017800018520004700370083c7b300cd
:1049500002fe2f000f014100f88057000a00780086
:1049600045fd0700b2ff37000b8144008d80fb003e
:104970008c01780000fe2f000f0040003bfe070076
:104980003c0037008d80fb000c01780000fe2f00fa
:104990000f004000e10007000000e0003500320099
:1049a00018007800000ce8009041780002fe2f000b
:1049b0000f014100f88057000a007800b1fe07009f
:1049c0009bff370000c8b30080cf560029003a0093
:1049d000180ce8001c80e900000e780010407800f8
:1049e000e0df9f0013002000e2fd2f000f014100d7
:1049f0000800370000c8b30080cf56001d003a0001
:104a0000180ce8001c80e900000e78008001eb0023
:104a100010017800f88057000a00780070fc070049
:104a200083ff370000c8b30080cf560011003a0062
:104a3000180ce8004fb29700efb19700080037005c
:104a40000e0c78000000eb00c0b79f00e0b79f009d
:104a50000080eb00d0b79f000002eb0084017800db
:104a600012002000618520000a0078004afe07003d
:104a70006fff3700180ce800090078004f07780036
:104a80004f06be004f05be004f04be006f01b100cf
:104a9000000006008200fa00889fbe008a1f78008e
:104aa0000005780082047800c13f9f000004eb00fd
:104ab000100037000902780088017800a2f72f0063
:104ac0000f01410081f72f008f8040000a0078001d
:104ad00084fe070008004000880f500004003d00dd
:104ae000b0042000704388000084eb00040037000d
:104af000000478004f3897001004e000edff3a0002
:104b0000080078004f0578004f04be000080fa00ce
:104b10000000060080007800100020000202200043
:104b2000828f500004003200e9805000e48f500072
:104b3000010036000000eb0000000600889fbe0068
:104b40008a1f7800000578000a04780098447800ed
:104b50000805e8000900fb00eeff07000000e00088
:104b6000f9ff3a00b0c2b30080cf54000500320014
:104b7000d0c2b3008000eb0080cf540005003a00a3
:104b8000020037008000eb00010037001100200018
:104b90000804e8000000eb00030037006a02b900d7
:104ba000020052000003b0003801fb0003fd2f009b
:104bb00082814100e98f5100f8ff36000100e000da
:104bc00001003a000000ea004f0578004f04be00e3
:104bd000000006008001780002003700b15978001b
:104be0000201e9000200e000fcff3a0000000600bc
:104bf00080007800040037003104e00002003a0031
:104c00000000510000000600010178000108a30027
:104c1000f9ff3a008101780031017800f4ef2f00ac
:104c2000020242000281ea00020162000408280038
:104c300004016100f7ff3200830078000101780071
:104c40003104e000fdff3a000000510000000600c2
:104c5000f1fb2f0080804000f98f500001003e00e2
:104c60000050a00000000600f9ff3700f1f92f0006
:104c700080804000f98f500001003e00f005b20036
:104c800000000600f9ff3700f28747008e1f78000a
:104c900002027800030178000000e0000200320008
:104ca0000007780001003700728757008002eb0090
:104cb0000100e000010032008102e900708057002d
:104cc000060009000018eb000080eb0080bf9f0089
:104cd0002310200093bf9f00aebf9f00b1bf9f0075
:104ce000c5bf9f000100e00003003d00b1042000ab
:104cf0007143880006003700004feb00eebf9f00b5
:104d0000debf9f00840078007080570022000700fb
:104d10004f0778002f01b10000000600881f7800bf
:104d20000004780000082000808f50001700350034
:104d300010082000808f50000b0034003008200045
:104d4000808f500011003a00920078006880500077
:104d5000000978003002be002003be00049cbe00a3
:104d60000694be000700370092027800648052006b
:104d7000000978001000be0015000700009cbe006e
:104d80000294be0010002000010037000000eb007c
:104d90004f047800000006000200fa00881f780027
:104da00000047800e2bf9f0064815700080078008b
:104db00038ff0700980090000148a300010032006e
:104dc0000080eb004f0478000080fa00000006002d
:104dd000810378001d0007000001be006000b800dc
:104de0000478a30013003a006220e10015003e00a1
:104df0000d0039008301d1000281d3008180d300ee
:104e00008301d1000281d3008180d3008301d100ce
:104e10000281d3008180d3000538b000c42add00b0
:104e2000f300b2008381720007f0a70003f0a00036
:104e30000000060083ff2700020020006110b90077
:104e4000f9ff370003ff2700f7ff3700c70ade002e
:104e5000f107b200f50fb20008003200e1cf4200c6
:104e6000020032000170a00024000500810f7000d4
:104e7000010032000408050044000500810f7000a5
:104e800002003a00140005008502e900000040001d
:104e900081c04800fcff3b000170a0002400050019
:104ea000020ab900001bb9000200b80081004200ec
:104eb0008100430000000600889fbe008a9fbe005c
:104ec00030044200b0844a0030054b0090854b000e
:104ed0006000b1000898be000a90be000440e100e6
:104ee00005c8e10006d0e10007d8e100020031006a
:104ef000680040001008e8004f05be004f04be00e7
:104f000000000600889fbe008a9fbe003004be00dd
:104f10002005be000418540005985c0006185d00ca
:104f200007985d00110020000440e10005c8e10081
:104f300006d0e10007d8e100010039008000eb0055
:104f4000108810004f05be004f04be000000060090
:104f50001200fa00889fbe008a9fbe008c9fbe0090
:104f6000e0b79f00f1b79f0082bf9f0093bf9f00f3
:104f70000605be000404be000000eb00d0b79f0091
:104f8000c0b79f00b0b79f00a0b79f0090b79f0029
:104f9000000678005fb19700cfb097008201410012
:104fa0003fb097000200e00004003d00370007001a
:104fb0007e805700c0ff0700030037003300070062
:104fc0007e805700cfff0700dfb697000d00e0009e
:104fd0000c0035006fb29700ffb297000fbb97002f
:104fe0009fbb970010002000010020006011b80056
:104ff00000027200818272000203730083837300d7
:105000001b0007000c06e80001042000810f560079
:10501000e0ff3a000d00e00004003d000802be0081
:105020000a03be007e805700a3ff07005fa8970019
:105030000000e00005003a001fb29700afb29700f1
:105040003fb39700cfb39700090007006fb09700f8
:10505000ffb097000fb997009fb997004f06be00a9
:105060004f05be004f04be000080fa00000006009d
:105070000100070000000600a4b79f00b5b79f001d
:10508000c6b79f00d7b79f00000006004f09de009b
:1050900082817100b3b79f004f01de008180400024
:1050a00082807000a1b79f008fb097004f09de008b
:1050b000000040000200700090b79f007fa897009a
:1050c0004f01de00818040008280700081b79f0028
:1050d0000d0007004f3ade000000400004007000a1
:1050e000f0af9f00080007000402420085824a00da
:1050f00006034b0087834b00dfff07000802be005a
:105100000a03be00000006002fb29700bfb297004e
:105110004fb39700dfb3970000000600881f7800a8
:1051200018002000881f780089ff07008f87e9009a
:105130004f04780000000600801feb0084ff07008a
:105140008f87e90000000600889fbe008a9fbe008e
:10515000e00f5000e08f5800e00f5900e08f590039
:105160000c003d006044b8006055b80000005400d9
:1051700081805c0002015d0083815d0018002000d9
:105180001500070008003d00180007000004eb00b0
:10519000050037000004eb000f00070002003d008f
:1051a0001200070018002000dcff07000800e000e4
:1051b000060032006022b8006033b80000005200e0
:1051c00081805a0002015b0083815b004f05be00b5
:1051d0004f04be0000000600e00f5200e08f5a00ae
:1051e000e00f5b00e08f5b00000006006044b80049
:1051f0006055b8000402540085825c0006035d001f
:1052000087835d0000000600889fbe008a9fbe0065
:105210008c1f7800e00f5000e08f5800e00f59001d
:10522000e08f59000d003d006044b8006055b800a3
:105230000000540081805c0002015d0083815d00fc
:105240001c0020000820e10009a8e1000ab0e100ec
:105250000bb8e1000d003d00080037000006eb0030
:10526000e00f5200e08f5a00e00f5b00e08f5b0020
:1052700006003d006044b8006055b80004025400c8
:1052800085825c0006035d0087835d00aaff07003e
:105290000c00e000060032006022b8006033b80065
:1052a0000000520081805a0002015b0083815b0094
:1052b0004f0678004f05be004f04be0000000600f8
:020000040000fa
:1052c000020400000e0100000f1100000f0000009a
:1052d000020400000e1100001f1000000e0000006c
:1052e000020400000c040000040400000e00000092
:1052f000020400000e110000111100000e00000059
:105300000204000011110000111300000d00000044
:105310000a00000011110000111300000d00000030
:10532000050a000011110000111300000d0000001b
:10533000050a00000e110000111100000e0000000f
:105340005246000049440000204300006172000002
:105350006420000052650000616400006572000076
:10536000002000002025000030330000690000000c
:020000040000fa
:105370000000fa002022ef002222ef00f0192000a6
:10538000401188002062a80021e2a8002342a80062
:105390000080fa00000006000200fa00000f78000a
:1053a000000000001111800000202000008060003b
:1053b0000000e000fbff3a001e007800201188008a
:1053c0001e0078000080fa00000006000200fa00cb
:1053d000000f7800050037001e00780010407800ac
:1053e0000000fb001e0fe800ebff07001e00780026
:1053f000104078000004e000f7ff3a000080fa0057
:10540000000006000000fa000000000010118000fb
:10541000610060000000e000fcff320030118000fd
:10542000004078000080fa00000006000600fa0044
:1054300010079800210798009e009000010f780047
:10544000f0ff07009e009000804878001e0090004a
:10545000104078000000fb00cfff07001e00900006
:105460000000e800100798002e0090000000e900fe
:10547000200798002e009000e10f5000f0ff3c0044
:105480001e0090008040eb00014878001e0078006c
:105490000080fa00000006001200fa00213a8000a5
:1054a000f0f32f0000806000203a880001003700f0
:1054b00000000000113a800000022000008060001f
:1054c0000000e000faff320040a7a900113a800076
:1054d000f00b2000008160006004200071052000b6
:1054e000237420008049780081497800824978003f
:1054f0002135800000fc2f00008060008001b30097
:1055000020358800b1368000f00f2c0080806000cc
:105510000030200001007000b0368800103a800092
:10552000000178000260a0006004200071052000e6
:1055300023742000804978008149780082497800ee
:10554000f0c2a900f0e2a900f102a900f122a9002d
:10555000d9e2a900e882a900e8a2a900d022a80007
:10556000d062a800e102a800e122a80078000700ac
:10557000e0000700009a2a008e0007000e80e80075
:10558000f200200001022000a3f8070078ff0700c6
:105590000000eb00000f78000000000099ff0700fa
:1055a000e24f5000fdff3a000e80e800c1002000ed
:1055b0009eff07000000000092ff0700e34f50002d
:1055c000fdff3a00e01680000080ea004f00de0098
:1055d000004078000080fb004f00dd00e1168000f5
:1055e00001f0a10001007000e01688001e0fe80025
:1055f0008040eb0000ccb3002b0007000e80e800d9
:105600006c0007009e1f7800109b2a00801f780006
:105610000080200073f80700e48757000080200016
:105620006400070000000000dcff37000000fa0003
:10563000ec22a800000000000000000000000000b4
:10564000ec22a9000080fa00000006000000fa0029
:105650000117800000f02f00008060000017880014
:10566000f002a900f022a900e822a900f402a90092
:10567000f422a900ec22a9000080fa000000060034
:105680000200fa00004f78002117800000f02f0080
:10569000808060001e00fb00010070002017880061
:1056a0000080fa00000006000400fa00204798007d
:1056b0003147980001178000f00f200001007000b2
:1056c00000178800f422a800f402a900ec22a80028
:1056d0000000000000000000000000001017800023
:1056e0004700de0061406000004f7800ec22a90016
:1056f0001e4078000004e000f4ff3a00011780002b
:1057000000f02f000080600000178800f422a9003c
:105710003e4090000080fb000000ea004f00de00e9
:10572000004078000080fb0061006000a11780004d
:105730000100a10001007000a01788002e40900019
:10574000cfff0700b9ff07000080fa000000060045
:105750000000fa00bdff070000202100a107200083
:105760008e0007008040eb0080c3b300ceff07002f
:105770008040eb0080c0b300cbff07008040eb000f
:1057800010c0b300c8ff07008040eb0060c0b3004a
:10579000c5ff07008040eb00c0c0b300c2ff070098
:1057a00000b82b00010020007c0007000080fa00f8
:1057b000000006000400fa001007980047003700b8
:1057c0001e009000104f78001e00fb00eb0f400001
:1057d0002f003200eb0f40000c003c00f70f4000a0
:1057e00019003200f70f400003003c00ff0f40009b
:1057f000120032002c003700f30f40001500320079
:10580000ed0f40001600320027003700e60f400081
:1058100016003200e60f400003003c00ea0f400093
:105820001e00320020003700e50f40001500320056
:10583000e40f4000100032001b0037000040eb0076
:10584000004f78001800370010c0b300004f7800f8
:105850001500370020c0b300004f78001200370059
:1058600030c0b300004f78000f00370040c0b300d5
:10587000004f78000c00370050c0b300004f780094
:105880000900370060c0b300004f78000600370001
:1058900070c0b300004f780003003700f0ceb300b3
:1058a000004f7800000000001e407800ea4f5000d2
:1058b00004003a008040eb0000ccb3007aff070000
:1058c000030037001e40780011c0b30076ff0700c8
:1058d0001e0090000000e800100798001e009000d5
:1058e000104078000004e000b5ff3a000080fa00a4
:1058f000000006000200fa008040eb0000c4b30084
:1059000069ff07000000eb00000f78000600370079
:1059100000962a001e0040001040780011c0b3001d
:1059200061ff07001e0fe800f00320009e007800d2
:10593000808f5000f6ff34008040eb0000c8b300b9
:0c59400059ff07000080fa00000006007c
:020000040000fa
:10594c00000800005000000000000000500800009b
:10595c001e00000002000000286e69006c29000087
:10596c0025006800076c09004c836a009074a00045
:10597c007ac000008068880000846c00820081007e
:10598c006e08000002000000000000000000000093
:020000040000fa
:10599c00f03fb1000180b10006003500ee030900b4
:1059ac0000000000403fb1000180b100fbff3d0052
:1059bc001000b000203fb00002003500008009004c
:0859cc000000000000000600cd
:020000040000fa
:020000040005f5
:0457f400ffff0000b3
:020000040000fa
:020000040005f5
:0457f800b6230000d4
:020000040000fa
:020000040005f5
:0457fc006f3e0000fc
:00000001FF
